:100000000C94B8010C94D5010C94D5010C94D50135
:100010000C94D5010C94CC040C94D5010C94D5010E
:100020000C94D5010C94D5010C94FC040C94D501CE
:100030000C94D5010C94D5010C94FB040C94FB0496
:100040000C94FA040C94D5010C94D5010C94D501B0
:100050000C94D5010C9423060C94D5010C94D50175
:100060000C94D5010C94D501467265712020562F51
:10007000487A2020416D7020005020202049202007
:1000800020442020202044542000526561642044F4
:100090006F6E652020202020202000526561646959
:1000A0006E6720454550524F4D20200046726571C5
:1000B0002020562F487A2020416D7020005646207F
:1000C0004D6F746F722044726976650A0053746FC5
:1000D00072656420202020202020202020005374DE
:1000E0006F72696E6720454550524F4D2020004584
:1000F0006E646520646572204661686E656E737417
:10010000616E676500312E31202863293230303925
:100110002D32303137206D61747A6574726F6E697B
:1001200063730000000000000000060004080D00DA
:1001300000DD0800E11100E51900E82100EC2A00CB
:10014000EF3200F13A00F44200F64A00F85200FAA9
:100150005A00FC6200FD6900FE7100FE7800FF801D
:1001600000FF8700FF8E00FE9500FE9B00FDA200B1
:10017000FCA800FAAE00F8B400F6BA00F4C000F132
:10018000C500EFCA00ECCF00E8D400E5D900E1DDFE
:1001900000DDE100D9E500D4E800CFEC00CAEF00B3
:1001A000C5F100C0F400BAF600B4F800AEFA00A839
:1001B000FC00A2FD009BFE0095FE008EFF0087FF65
:1001C000007FFF0078FE0071FE0069FD0062FC0008
:1001D0005AFA0052F8004AF60042F4003AF10032AE
:1001E000EF002AEC0021E80019E50011E10008DD2C
:1001F0000000E10800E51100E81900EC2100EF2AF9
:1002000000F13200F43A00F64200F84A00FA5200D7
:10021000FC5A00FD6200FE6900FE7100FF7800FFDD
:100220007F00FF8700FE8E00FE9500FD9B00FCA274
:1002300000FAA800F8AE00F6B400F4BA00F1C0006D
:10024000EFC500ECCA00E8CF00E5D400E1D900DD3D
:10025000DD00D9E100D4E500CFE800CAEC00C5EF2D
:1002600000C0F100BAF400B4F600AEF800A8FA003D
:10027000A2FC009BFD0095FE008EFE0087FF008023
:10028000FF0078FF0071FE0069FE0062FD005AFC6D
:100290000052FA004AF80042F6003AF40032F10047
:1002A0002AEF0021EC0019E80011E50008E1000048
:1002B000DD0000E10800E51100E81900EC2100EF85
:1002C0002A00F13200F43A00F64200F84A00FA52ED
:1002D00000FC5A00FD6200FE6900FE7100FF78001C
:1002E000FF8000FF8700FE8E00FE9500FD9B00FC56
:1002F000A200FAA800F8AE00F6B400F4BA00F1C00B
:1003000000EFC500ECCA00E8CF00E5D400E1D90059
:10031000DDDD00D9E100D4E500CFE800CAEC00C57E
:10032000EF00C0F100BAF400B4F600AEF800A8FA8D
:1003300000A2FC009BFD0095FE008EFE0087FF00E2
:1003400080FF0078FF0071FE0069FE0062FD005A28
:10035000FC0052FA004AF80042F6003AF40032F18A
:10036000002AEF0021EC0019E80011E50008E10087
:1003700011241FBECFEFD8E0DEBFCDBF11E0A0E05B
:10038000B1E0E2EEF3E102C005900D92A032B107B8
:10039000D9F721E0A0E2B1E001C01D92AD33B20770
:1003A000E1F70E942B070C94EF090C940000CF9307
:1003B000DF93DC01FB01E9011A821B821C821D8292
:1003C000198218829F838E83798768875B874A8723
:1003D0008FEF9FE7BD010E9412097D876C879F0107
:1003E000FF0F440B550B61E070E08FEF9FE70E9419
:1003F00048092E873F87488B598BDF91CF9108950D
:10040000EF92FF920F931F93CF93DF938B01FA012B
:100410009C01261B370B848595858217930784F0F2
:10042000919581959109281739076CF086819781FC
:10043000289FE001299FD00D389FD00D112405C0C1
:10044000CFEFDFE702C0C1E0D0E8C901330FAA0B4C
:10045000BB0B42815381648175819A01AB01280FE6
:10046000391F4A1F5B1F86859785A089B18982172E
:100470009307A407B5074CF482839383A483B583C1
:1004800061E070E08FEF9FE71DC0B095A09590955B
:1004900081959F4FAF4FBF4F281739074A075B071A
:1004A0004CF482839383A483B5836FEF7FEF80E066
:1004B00090E808C02283338344835583A085B185A7
:1004C0000E94760920813181201B310BA285B385E2
:1004D0002A9F70012B9FF00C3A9FF00C112411837E
:1004E00000838E01DD0F220B330BAB01BC01400FEB
:1004F000511F621F731FC701FF0CAA0BBB0B8A01A0
:100500009B01080F191F2A1F3B1FC901B80120E0DA
:1005100031E040E050E00E944809213010E8310706
:100520001FEF4107510724F421E030E84FEF5FEF60
:10053000DA01C901811520E89207A105B10524F06F
:100540008FEF9FE7A0E0B0E0DF91CF911F910F9177
:10055000FF90EF900895FC0112821382148215829D
:10056000089584B1817F84B98AB187798AB9089561
:10057000CF93C82FE82FE295EF70F0E0E45FFE4FD5
:1005800080810E94C406CF70EC2FF0E0E45FFE4F44
:100590008081CF910C94C406CF93C82F892F0E94DD
:1005A000B8028C2FCF910C94B80280E20C94C40650
:1005B000DF92EF92FF920F931F93CF93DF934AE066
:1005C00060E071E00E94890980933C01E0E0F1E085
:1005D00001900020E9F73197E050F140DE2E80E0F5
:1005E000E82E81E0F82E8701FF27EF012197802F69
:1005F0008E198D1578F4C801805091408C179D0795
:1006000019F48EE20E94C406F80181918F010E94C4
:10061000C406EDCFDF91CF911F910F91FF90EF9026
:10062000DF900895DB01FA0190911E01981710F0F8
:100630001C921AC090911E01482F50E02FEF30E01D
:10064000291B3109421753073CF080911E01880F86
:1006500080958C938FEF08C090911E01282F291B45
:100660002C9390911E01890F8083089589B1809504
:100670008770089561E080E00E94B3068EED90E0FF
:100680000E94E406F8940E94B102F999FECF6091AD
:100690001E0188E090E00E94CC09F999FECF682DF8
:1006A00087E090E00E94CC09F999FECF672D86E0A3
:1006B00090E00E94CC09F999FECF60912D017091D4
:1006C0002E0184E090E00E94DA09F999FECF609152
:1006D0002F017091300182E090E00E94DA09F999CF
:1006E000FECF609131017091320180E090E00E9474
:1006F000DA09F999FECF292D2C60922E78948FEF8C
:1007000099E628E1815090402040E1F700C00000C8
:1007100061E080E00E94B3068DEC90E00E94E40668
:100720008FEF99E628E1815090402040E1F700C02A
:1007300000000C943603EF92FF920F931F93CF9318
:10074000DF930E94C10689E790E00E94E4061092C0
:1007500022010E9436038111FCCFD0E088ECF82EF4
:1007600001E010E098E0E92E0E943603C82F8330A4
:1007700009F4A5C028F4813059F08230B1F006C0E8
:10078000843009F45CC0853009F49BC0D0E099C086
:10079000809122018F5F8093220180912201843019
:1007A00008F48FC0109222018CC080912201813008
:1007B000B9F028F0823029F18330A1F182C0809114
:1007C0002D0190912E011816190624F010932E0178
:1007D00000932D0180912D0190912E01019742C02F
:1007E00080912F01909130011816190624F0109372
:1007F000300100932F0180912F01909130010197DA
:100800003FC080913101909132011816190624F0F1
:1008100010933201009331018091310190913201A6
:1008200001973CC080911E01815080931E018091F0
:100830001E01883008F045C0E0921E0142C0809140
:1008400022018130A1F028F08230F9F0833059F193
:1008500038C080912D0190912E0180912D019091B1
:100860002E01019690932E0180932D012AC0809134
:100870002F019091300180912F01909130010196CC
:100880009093300180932F011CC080913101909191
:1008900032018091310190913201019690933201A1
:1008A000809331010EC080911E018F5F80931E01E5
:1008B00080911E01893C28F0F0921E0102C00E9426
:1008C0003A03409131015091320160912F017091B2
:1008D000300180912D0190912E0127E231E00E949C
:1008E000D7010E9436038823A1F0DF5FDA3050F48D
:1008F0002FEF8DEE92E0215080409040E1F700C054
:10090000000007C08FE39CE90197F1F700C00000E9
:10091000DBE061E080E00E94B30680912D019091C0
:100920002E010E94CC0280912F01909130010E94F3
:10093000CC0280913101909132010E94CC020E9440
:10094000D50280911E010E94B8020E94D502E0915A
:100950002201F0E0E55DFE4F849161E00E94B30664
:100960008FE19EE40197F1F700C00000C53009F067
:10097000FBCE109222010E94BE0688E690E00E9403
:10098000E4060E9436038111FCCFDF91CF911F91C5
:100990000F91FF90EF9008951F920F920FB60F9254
:1009A00011242F933F934F935F936F937F938F9374
:1009B0009F93AF93BF93EF93FF9389B18095881F67
:1009C0008827881F80FB91F80E94B102892D8C60D6
:1009D000982EFF91EF91BF91AF919F918F917F9151
:1009E0006F915F914F913F912F910F900FBE0F909C
:1009F0001F901895189518951F920F920FB60F9289
:100A00001124CF92DF92EF92FF920F931F932F93B7
:100A10003F934F935F936F937F938F939F93AF9386
:100A2000BF93EF93FF93CF93DF9300D0CDB7DEB7A3
:100A3000892D869586958370813011F10E94B102CF
:100A400081EB84BD92EB909380008093B000109274
:100A5000B3001092880017BC8FEF8093B40080938E
:100A60008A0088BD80E286BBB59BFECF892D837F3F
:100A70008460982E84B18E6084B98AB188668AB900
:100A8000882D90E01C012091390130913A01820FAC
:100A9000931F90933A01809339018091390190918D
:100AA0003A018115904C48F08091390190913A01BA
:100AB000905C90933A018093390180913901909133
:100AC0003A01892F9927FC01EE0FFF1F8E0F9F1F00
:100AD000FC01E15DFE4F8F010F5F1F4F2491CF019D
:100AE0000296F80191FC04C00491FC01E49003C05B
:100AF000E490FC010491629E900111246E9C7001AF
:100B00001124609E80011124AE014F5F5F4FBE0132
:100B10006E5F7F4F832F0E9412038A8187BD898178
:100B200088BDAE014F5F5F4FBE016E5F7F4F8F2D5F
:100B30000E9412038A8180938800898180938A00B1
:100B4000AE014F5F5F4FBE016E5F7F4F812F0E94EE
:100B500012038A818093B30089818093B4008091CD
:100B600023018F5F80932301883C08F451C090FEDD
:100B700016C020913B01C0903B01E82DF0E030E031
:100B8000AFEFB0E00E946709BB27A92F982F872FEE
:100B900047E251E0BF010E9400028C0D882E682DB3
:100BA00070E080E09BE40E94FE089B0140E050E082
:100BB00066ED7CED81E090E00E94260930932601ED
:100BC00020932501C9016AE070E00E94FE08769E2C
:100BD0009001779E300D1124B90180E090E0232B25
:100BE00059F0663FF9E07F078105910544F066EF13
:100BF00079E080E090E003C060E070E0CB012AE0A3
:100C000030E040E050E00E944809622E109223013B
:100C10000F900F90DF91CF91FF91EF91BF91AF9126
:100C20009F918F917F916F915F914F913F912F9104
:100C30001F910F91FF90EF90DF90CF900F900FBE1C
:100C40000F901F90189578941F920F920FB60F92E5
:100C500011242F938F939F9390FE22C080917C004C
:100C6000843659F08536B1F48091790090E0870D93
:100C7000911D95958795782E0DC020913B0180910F
:100C8000790090E0820F911D9595879580933B01A7
:100C900085E601C084E680937C008EED80937A0027
:100CA0009F918F912F910F900FBE0F901F901895CD
:100CB000289A00C0289808951F93CF93DF931F921E
:100CC000CDB7DEB7662311F02C9A01C02C985C9842
:100CD00097B19F6097B998B1192F107F982F92956F
:100CE0009F70912B98B989830E94580689818F70D3
:100CF000812B88B90E9458061F6018B90F90DF91A8
:100D0000CF911F9108952C985C9A87B1807F87B905
:100D1000289A00C096B1289800C0289A00C026B131
:100D20002F70892F8295807F2898822B08950E94AA
:100D3000830687FDFCCF88E090E00197F1F70C94E3
:100D40008306CF93C82F0E94970660E08C2FCF9127
:100D50000C945C06CF93C82F0E94970661E08C2FFD
:100D6000CF910C945C06611102C0805801C0805480
:100D70000C94A1060E94970690E0089581E00C94DF
:100D8000A10682E00C94A106CF93C82F0E9497067B
:100D9000CA3049F4803410F080E001C080E480580B
:100DA000CF910C94A10661E08C2FCF910C945C063E
:100DB000CF93DF93EC018991882319F00E94C40638
:100DC000FACFDF91CF910895CF93DF93FC01849107
:100DD000EF012196882321F00E94C406FE01F7CF7F
:100DE000DF91CF9108951F93CF93DF93182F97B181
:100DF0009F6097B9249A549A209AE0E0FAEF3197CD
:100E0000F1F7419A409A0E945806E0E0FEE43197DB
:100E1000F1F70E945806C0E0D1E0FE013197F1F7EA
:100E20000E945806FE013197F1F740980E9458063B
:100E30002197F1F788E20E94A10688E00E94A106AE
:100E40000E94BE0686E00E94A106812FDF91CF910D
:100E50001F910C94A106F894612C10923B018824F8
:100E60008394109222018FE087B985B1817F85B983
:100E70008BB187798BB92D9A8AB1887F8AB9259AE7
:100E80008BB187688BB98CE00E94F3060E94C10683
:100E90008DEB90E00E94E40680E30E94C40681E0AE
:100EA00084BD92E0909380008093B0002FEF30E0FB
:100EB000309387002093860016BC23E030E0309307
:100EC00085002093840095E09093B20085BD91E168
:100ED000909381008093B10081E30E94C40680E872
:100EE00080936D0084E08093680082E30E94C406D2
:100EF00086E980937A0080E380937E0084E6809385
:100F00007C0010927B0086EC80937A000E94B102F4
:100F10002FEF83EC99E0215080409040E1F700C032
:100F200000008EED80937A0083E30E94C40627E2DE
:100F300031E040E150E068E070E080E690E00E943F
:100F4000D70184E30E94C406E89490F8E89491F8ED
:100F5000E92DEC609E2E85E30E94C40689B1809540
:100F6000881F8827881F80FB91F8689490F887E293
:100F700086BB80E280936F0086E30E94C406FFEF89
:100F800029E688E1F15020408040E1F700C00000F0
:100F900061E080E00E94B3068BE990E00E94E406E5
:100FA00088E090E00E94BE0980931E0180911E019E
:100FB000883018F488E080931E0187E090E00E945A
:100FC000BE09882E86E090E00E94BE09782E84E05B
:100FD00090E00E94C60990932E0180932D0182E03B
:100FE00090E00E94C6099093300180932F0180E029
:100FF00090E00E94C60990933201809331019FEFE7
:10100000E9E6F8E19150E040F040E1F700C000006F
:1010100061E080E00E94B3068AE890E00E94E40666
:101020002FEF89E698E1215080409040E1F700C021
:1010300000000E94360387E30E94C4060E94BE0699
:101040008EE00E94A1068CEA90E00E94E40678946B
:101050000BE0CFEFD0E00E94360390FC41C082301D
:10106000B9F018F4813039F052C0833009F44CC023
:10107000843009F14CC0809122018F5F809322015E
:1010800080912201823008F444C01092220141C0B4
:1010900080912201882319F0813039F03AC0811003
:1010A00002C0882483948A9434C0711002C07724CB
:1010B00073947A942EC080912201882319F0813094
:1010C00041F027C0EFEF8E1202C02EEF822E8394E4
:1010D00020C0FFEF7F1202C09EEF792E739419C0DB
:1010E000813019F0833081F012C09091200181E0AD
:1010F000911180E08093200180912001882311F0DC
:101100002D9807C02D9A05C00E949B0302C0109223
:1011100024010E9436038823C9F0809124018F5F47
:10112000809324018A3050F42FEF8DEE92E021500D
:1011300080409040E1F700C0000008C0EFE3FCE908
:101140003197F1F700C000000093240161E080E0D6
:101150000E94B30680912501909126010E94D80239
:101160000E94D50261E086E00E94B306872D90E0E0
:101170000E94D8020E94D5020E94D50261E08CE054
:101180000E94B306F4E66F9EC0011124BE010E94C6
:10119000FE08CB014AE060E071E00E94890980937B
:1011A0003C01E0E0F1E001900020E9F73197E050E8
:1011B000F1401E2F80E0E82E81E0F82E67018C2D93
:1011C0008E19811730F4F60181916F010E94C406D7
:1011D000F6CF85E20E94C4060E94D502E09122016A
:1011E000F0E0E75DFE4F849161E00E94B3068FE17D
:1011F0009EE40197F1F700C000002DCFAA1BBB1B96
:1012000051E107C0AA1FBB1FA617B70710F0A61B06
:10121000B70B881F991F5A95A9F780959095BC0127
:10122000CD01089597FB072E16F4009407D077FDA3
:1012300009D00E94FE0807FC05D03EF490958195E8
:101240009F4F0895709561957F4F0895A1E21A2EE2
:10125000AA1BBB1BFD010DC0AA1FBB1FEE1FFF1F5A
:10126000A217B307E407F50720F0A21BB30BE40BAA
:10127000F50B661F771F881F991F1A9469F76095F1
:101280007095809590959B01AC01BD01CF010895AB
:10129000052E97FB1EF400940E945F0957FD07D0AE
:1012A0000E94260907FC03D04EF40C945F09509568
:1012B0004095309521953F4F4F4F5F4F0895909542
:1012C0008095709561957F4F8F4F9F4F0895A29F96
:1012D000B001B39FC001A39F700D811D1124911D0A
:1012E000B29F700D811D1124911D0895B7FF0C94BC
:1012F0007E090E947E09821B930B08950E94670954
:10130000A59F900DB49F900DA49F800D911D112459
:101310000895BB274A3031F4992322F4BDE2909519
:1013200081959F4F0C949509BB27FB015527AA2750
:10133000880F991FAA1FA41710F0A41B8395505162
:10134000B9F7A05DAA3308F0A95DA193009779F7DA
:10135000B111B1931192CB010C94AE09DC01FC01E7
:10136000672F71917723E1F7329704C07C916D93D9
:1013700070836291AE17BF07C8F30895F999FECF45
:1013800092BD81BDF89A992780B50895A8E1B0E093
:1013900042E050E00C94E109262FF999FECF1FBAE4
:1013A00092BD81BD20BD0FB6F894FA9AF99A0FBE8E
:1013B000019608950E94CC09272F0C94CD09DC01D9
:1013C000CB01FC01F999FECF06C0F2BDE1BDF89A50
:1013D000319600B40D9241505040B8F70895F894FA
:0213E000FFCF3D
:1013E20030303030303030303030303030313233F5
:1013F20034353637383941424344454600001400FB
:00000001FF
